:02000000822854
:1000080064000C1E0428990003147D2800308A001F
:1000180028080739820701340234043408341034BC
:10002800203440348034A301A200FF30A207031C0F
:10003800A307031C7D280330A100E43025201928DC
:10004800A101F63EA000A109031C3028FE300000E3
:10005800A00703182B28A0076400A10F2A28000076
:1000680020183628201838280800A8000A20A001DF
:10007800A101A81DA000A819A10020087D2803102F
:10008800A10CA00CFF3E0318432820087D28A501D9
:10009800A4011030A600210DA40DA50D2208A4026C
:1000A8002308031C230FA502031861282208A407AC
:1000B80023080318230FA5070310A00DA10DA60BF5
:1000C8004F2820087D281030A800A101A001A70C06
:1000D800A60C031C75282208A00723080318230F61
:1000E800A107A10CA00CA50CA40CA80B6B28240834
:1000F8007D288313031383126400080083160730D6
:1001080099002030980083129030980083160730A9
:100118009F00811783128611831686110710871096
:100128000711071287128312B030DE001030C100A9
:10013800C0014030C70083168601831287168316D4
:1001480087128312871083168710831287108316ED
:100158008710C83083128A011720871483168710E6
:1001680083128714831687108312871283168712C7
:10017800533083128A01042074308A0104206130CC
:100188008A01042072308A01042074308A01042014
:1001980069308A0104206E308A01042067308A01A0
:1001A80004202E308A0104202E308A0104202E30AB
:1001B8008A0104200D308A0104200A308A010420B3
:1001C8008A110A123F2C8710831687103230831247
:1001D8008A0124208714831687108312E230CC000A
:1001E8008A110A122021A230CC008A110A12202179
:1001F800A030CC008A110A122021C830CC008A1104
:100208000A1220212630CC008A110A1220218130BE
:10021800CC008A110A1220212030CC008A110A123F
:1002280020212F30CC008A110A122021AF30CC00B7
:100238008A110A1220210800071683160712831252
:1002480007118316071183128712831687128312E8
:1002580007108316071083124C08860007148316AC
:100268000710831287168316871283120800071651
:100278008316071283120715831607118312871234
:1002880083168712831207108316071083125008EB
:1002980086000714831607108312871683168712A1
:1002A800831208008316FF30860083120714831612
:1002B80007108312071183160711831287128316FA
:1002C8008712831207128316071283120608D300B7
:1002D800071683160712831287168316871286015C
:1002E80083120800B030DE006400B8305E028A1164
:1002F8000A120318A4294030CC008A0120215E0884
:10030800CC008A0120211030CC008A012021043041
:10031800CC008A0120210430C300640084304302E9
:100328008A110A1203189F298A013B21C30A8A11DC
:100338000A12031D9129DE0A8A110A12031D78295F
:100348000800D0018A01762108004030CC008A01DB
:1003580020215708A000A1010830A200A3018A01AA
:100368004B20B2002108B300B0303207DF005F082D
:10037800CC008A01202104305407DA005A08A00072
:10038800A10104308A014620B2002108B3001030D0
:100398003204CC008A0120210F305A05CC008A0192
:1003A80020214B08D0008A013B21080020303E0262
:1003B800BD00640050303E028A110A12031CE7296E
:1003C80050303E02BD003D08A600A7010530A2003E
:1003D800A3018A016720C5000130C8006400063007
:1003E80048028A110A120318132A640050303E0288
:1003F8008A110A12031C072A8A110A12F227C50A4F
:100408008A110A120B2A8A110A122826C50A8A0199
:10041800A921D40AC80A8A110A12031DF229D40A8A
:10042800CB018A01A92108005708A000A1010830C2
:10043800A200A3018A014B20B2002108B300B0300A
:100448003207DF005F08CC008A0120214030CC0051
:100458008A01202104305407DA005A08A000A101BB
:1004680004308A014620B2002108B300103032045B
:10047800CC008A0120210F305A05CC008A012021A6
:1004880008008A0118228316FF3086008312071499
:100498008316071083120715831607118312871214
:1004A800831687128312071283160712831206080F
:1004B800D100071683160712831207128316071234
:1004C80083120608D10007168316071283128716AF
:1004D800831687128601831208008A01452257086D
:1004E800A000A1010830A200A3018A014B20240822
:1004F800B2002508B30032088A013920D200510819
:100508005204CB008A01A92108008A014522570814
:10051800A000A1010830A200A3018A014B202408F1
:10052800B2002508B30032088A013920D2005108E8
:100538005206CB008A01A9210800D5014D08D80030
:100548000230A600A7014D08A200A3018A01672076
:10055800B2002508B3003208033CBA003308031C74
:10056800013E003CBB006400550858028A110A127B
:10057800031CFE2A8A110A12BB2364008A110A127C
:10058800BB1FDE2A0430A600A7015508A200A3015C
:100598008A016720B2002508B3000630B2070318A5
:1005A800B30A3208BA0733080318013EBB078A1199
:1005B8000A12FB2A58085502B200B301031CB30300
:1005C8000430A600A7013208A2003308A3008A015C
:1005D8006720B2002508B3000A30B2070318B30A2F
:1005E8003208BA0733080318013EBB07D803D50AF7
:1005F8008A01B72A0800D5014D08D8000230A600A4
:10060800A7014D08A200A3018A016720B2002508AE
:10061800B3003208033CBA003308031C013E003C17
:10062800BB006400550858028A110A12031C372BB4
:100638008A110A12BB230430A600A7015508A2009C
:10064800A3018A016720B2002508B3000630B2076B
:100658000318B30A3208BA0733080318013EBB0768
:10066800D50A8A01152B0800D5014D08D80002309B
:10067800A600A7014D08A200A3018A016720B200C5
:100688002508B3003208033CBA003308031C013EB6
:10069800003CBB006400550858028A110A12031C6A
:1006A800782B8A110A12BB2358085502B200B301ED
:1006B800031CB3030430A600A7013208A2003308C4
:1006C800A3008A016720B2002508B3000A30B207E8
:1006D8000318B30A3208BA0733080318013EBB07E8
:1006E800D803D50A8A014E2B0800D5014D08D80039
:1006F8000230A600A7014D08A200A3018A016720C5
:10070800B2002508B3003208033CBA003308031CC2
:10071800013E003CBB006400550858028A110A12C9
:10072800031CBA2B8A110A12BB2358085502B200BF
:10073800B301031CB3030430A600A7013208A200CA
:100748003308A3008A016720B2002508B3000A30E5
:10075800B2070318B30A3208BA0733080318013E70
:10076800BB070330D802D50A8A018F2B0800550829
:100778004E07D40058084F07D7008A017122550840
:100788004E02D40058084F07D7008A0171224E083C
:100798005507D40058084F02D7008A01712255081E
:1007A8004E02D40058084F02D7008A017122580817
:1007B8004E07D40055084F07D7008A017122580800
:1007C8004E02D4004F085507D7008A0171224E08FF
:1007D8005807D40055084F02D7008A0171225808DB
:1007E8004E02D40055084F02D7008A017122080032
:1007F8006400550856028A110A120318072C550876
:100808005602D507D6026400580859028A110A12FE
:100818000318122C58085902D807D9025508D400D1
:100828006400540856028A110A12031C282C58081E
:10083800D7008A0171225908D7008A017122D40A87
:100848008A110A12031D142C5808D700640057088F
:1008580059028A110A12031C3E2C5508D4008A0139
:1008680071225608D4008A017122D70A8A110A1205
:10087800031D2A2C08004C308A01042043308A01C9
:10088800042044308A01042020308A010420693081
:100898008A0104206E308A01042069308A0104200C
:1008A80074308A0104202E308A0104202E308A01F7
:1008B80004202E308A0104200D308A0104200A30D9
:1008C8008A0104208A01E7208A01A5210830D7007F
:1008D8001030D400E2016400123062028A110A1258
:1008E8000318A02C6208113C8A110A12031C992CC7
:1008F8008A110A128324BE008A110A12992C043024
:100908008A00620882074F34703474347234653454
:100918007834203446342D34353431343334323459
:10092800303420344C34433444348A01DA21E20A26
:100938008A110A12031D6F2C1030D7002430D400FE
:10094800E20164000B3062028A110A120318CF2CEC
:1009580062080A3C8A110A12031CC82C8A110A125E
:10096800B924BE008A110A12C82C04308A00620811
:1009780082074734723461347034683469346334BC
:1009880020344C34433444348A01DA21E20A8A118F
:100998000A12031DA52C1030D7000830D400E2013C
:1009A8006400083062028A110A120318FC2C6208DB
:1009B800073C8A110A12031CF42C8A110A12E82433
:1009C800CB008A110A12F42C04308A0062088207CC
:1009D800C334A534993481349934A534C3340034EC
:1009E800D40A8A01A921E20A8A110A12031DD42C09
:1009F8001030D7001430D400E201640008306202DD
:100A08008A110A120318292D6208073C8A110A1252
:100A1800031C212D8A110A121525CB008A110A12EE
:100A2800212D05308A0062088207183418341834DA
:100A380018347E34423424341834D40A8A01A92163
:100A4800E20A8A110A12031D012D1030D7006730FF
:100A5800D400E2016400083062028A110A12031805
:100A6800562D6208073C8A110A12031C4E2D8A1162
:100A78000A124225CB008A110A124E2D05308A002F
:100A880062088207263446348034903490348034A7
:100A980046342634D40A8A01A921E20A8A110A12A4
:100AA800031D2E2D1030D7007130D400E2016400F0
:100AB800083062028A110A120318832D6208073C63
:100AC8008A110A12031C7B2D8A110A126F25CB008A
:100AD8008A110A127B2D05308A0062088207FF34CA
:100AE8008134BD34A534A534BD348134FF34D40AEF
:100AF8008A01A921E20A8A110A12031D5B2D2030FE
:100B0800D7003C30D400E2016400083062028A1148
:100B18000A120318B02D6208073C8A110A12031C36
:100B2800A82D8A110A129C25CB008A110A12A82D19
:100B380005308A0062088207603460341F34033449
:100B4800C634FC3400340034D40A8A01A921E20AEC
:100B58008A110A12031D882D3030D7001830D400AE
:100B6800E20164000F3062028A110A120318E32DB1
:100B780062080E3C8A110A12031CDC2D8A110A1223
:100B8800C925BE008A110A12DC2D05308A006208C8
:100B9800820728346334293443344F344D34503475
:100BA8005334793473342034323430343034353477
:100BB8008A01DA21E20A8A110A12031DB52DD5012C
:100BC8007F30D600D8013F30D9008A01FC2302309B
:100BD800D5007D30D6000230D8003D30D9008A01DA
:100BE800FC231030CE002430CF000430CD008A0121
:100BF800A1220730CD008A01A1220A30CD008A0146
:100C0800A1222830CE008A0179235830CE008A01EB
:100C180038236F30CE008A01FF220430CD008A01CC
:100C2800FF220730CD008A01FF220A30CD008A0159
:100C3800FF224030CE002430CF000A30CD008A0198
:100C4800A12264008A01252E4508EF3C8A110A1268
:100C5800031CF12F8A110A123526CB008A110A12B9
:0A0C6800F12F07308A004508002F25
:100E000082070034003400340034003400340034ED
:100E10005F340034003400340734003407340034C5
:100E200014347F3414347F34143424342A347F341B
:100E30002A3412342334133408346434623436349C
:100E400049345534223450340034053403340034EA
:100E5000003400341C342234413400340034413432
:100E600022341C340034143408343E34083414342E
:100E7000083408343E3408340834003450343034F4
:100E8000003400340834083408340834083400349A
:100E900060346034003400342034103408340434B6
:100EA00002343E345134493445343E340034423403
:100EB0007F34403400344234613451344934463450
:100EC0002134413445344B34313418341434123421
:100ED0007F341034273445344534453439343C3478
:100EE0004A344934493430340134713409340534D6
:100EF00003343634493449344934363406344934B9
:100F0000493429341E340034363436340034003445
:100F10000034563436340034003408341434223467
:100F2000413400341434143414341434143400347C
:100F30004134223414340834023401345134093435
:100F4000063432344934793441343E347E341134F9
:100F5000113411347E347F344934493449343634C1
:100F60003E3441344134413422347F3441344134BD
:100F700022341C347F3449344934493441347F3479
:100F800009340934093401343E3441344934493494
:100F90007A347F340834083408347F3400344134E0
:100FA0007F34413400342034403441343F34013400
:100FB0007F3408341434223441347F344034403494
:100FC000403440347F3402340C3402347F347F3474
:100FD0000434083410347F343E34413441344134D5
:100FE0003E3408004508EF3C8A150A12031CF3281A
:100FF0008A110A12FF27CB008A150A12F32808303B
:101000008A00450882077F340934093409340634DC
:101010003E344134513421345E347F340934193440
:10102000293446344634493449344934313401345E
:1010300001347F34013401343F344034403440348F
:101040003F341F342034403420341F343F34403484
:10105000383440343F346334143408341434633443
:101060000734083470340834073461345134493457
:101070004534433400347F34413441340034023445
:1010800004340834103420340034413441347F3483
:101090000034043402340134023404344034403423
:1010A00040344034403400340134023404340034D9
:1010B000203454345434543478347F3448344434F1
:1010C00044343834383444344434443420343834A8
:1010D0004434443448347F343834543454345434ED
:1010E000183408347E340934013402340C34523458
:1010F000523452343E347F34083404340434783467
:10110000003444347D34403400342034403444349A
:101110003D3400347F3410342834443400340034F7
:1011200041347F34403400347C3404341834043483
:1011300078347C3408340434043478343834443417
:101140004434443438347C3414341434143408347F
:1011500008341434143418347C347C3408340434A3
:10116000043408344834543454345434203404346B
:101170003F344434403420343C3440344034203410
:101180007C341C342034403420341C343C3440340F
:10119000303440343C34443428341034283444341B
:1011A0000C345034503450343C344434643454346B
:1011B0004C34443400340834363441340034003480
:1011C00000347F3400340034003441343634083481
:1011D0000034103408340834103408347834463479
:1011E000413446347834080063008A150A12F42822
:02400E003D3D36
:00000001FF
